:020000040000FA
:0400000072303A28F8
:08000800A000030EA100831209
:100010008B1C32288B1031181428B11C3228643004
:10002000010203183128182800001628172818285C
:1000300019281A281B281C281D281E281F283110A3
:10004000B114A810031005190314AA0DA90DA80DC9
:10005000B00B322831152A08AF002908AE00280855
:10006000AD00B11081010B11210E8300A00E200EF6
:02007000090085
:0C007400203084008001840A6030040207
:10008000031C3C281230B00056218316FF23900039
:10009000831283160C308505870183128501870141
:1000A000073099000030831691009F008312C830FA
:1000B00083168100831231309000003083168C004B
:1000C000831210308B00742181018E018F010B117E
:1000D0008B100B108C018B177C20311992203A2148
:1000E000B30B7A28031085190314B90DF0303902C7
:1000F0000319E32075216C286400311808000B1DDA
:1001000008000B11B11031141230B000051D8D28FC
:10011000321483160113831208003210831601175C
:100120008312080031110130B7008B1320303707DC
:1001300083169B001C141A088312A400A500C0306B
:10014000A5061030370783169B001C141A0883126B
:10015000A3000030370783169B001C141A08831273
:10016000A2008B17321CBA2822090339A200A30966
:10017000A409A50922082D02031DDD2823082E024B
:10018000031DDD2824082F02031DCF28013037026C
:10019000031DCF283D18CF283D143E146E2125089D
:1001A0002F02031DDD2801303702031DDC283D1C12
:1001B000DC283D103E147121DD28B70A02303702D9
:1001C0000318080095280130B600B300B400B5004C
:1001D000B70085018701B1137C20B30B09290310F7
:1001E00085190314B90DF030390203193029B41FF1
:1001F0008501B41F8701B40B09293708B608031914
:10020000B60003190729FF3085008700B603963032
:10021000B400311DEC283111321C13292D0903398A
:10022000AD00AE09AF092F1CB1132F1CEC28B11B78
:10023000EC282E18EC28B1178B1320303707BB00A1
:100240002F08BA00432110303707BB002E08BA0030
:10025000432100303707BB002D08BA0043218B171C
:1002600085018701B70AB60102303702031CEC286A
:10027000742108003E1C08003E101030BB003D08F1
:10028000BA00432108008B133A0883161C159A0004
:100290003B089B0055309D00AA309D009C146400D3
:1002A0009C184F291C1183128B17080083161030DD
:1002B0009B001C141A088312BD00FF30D4000230CA
:1002C000D5000C30D600BA30D7003730D800DA303D
:1002D000D9006F30DA00B830DB0008000130BD0013
:1002E0000800850187010800080001303D05031959
:1002F00008005C180516DC1885165C190514DC1955
:1003000085145C1A8714DC1A07155C1B0714DC1BA8
:1003100087165D180716DD188715E6300E02031CD8
:100320009B290516851605148514871407150714CF
:100330008716071687158F08031908008F01850196
:1003400087015408DE002822D4005508DE00282248
:10035000D5005608DE00541C2822D6005708DE00BF
:10036000D41C2822D7005808DE00541D2822D800AB
:100370005908DE00D41D2822D9005A08DE00541E78
:100380002822DA005B08DE00D41E2822DB00CA0B1C
:10039000D1295408CA00D4185C14D41E5C10D41D92
:1003A0005C10CB0BDB295508CB00D51ADC14551D8E
:1003B000DC10551FDC10CC0BE5295608CC00561A72
:1003C0005C15561F5C11D61D5C11CD0BEF2957082B
:1003D000CD00571ADC15D71FDC11D71DDC11CE0B51
:1003E000F9295808CE00D81B5C16D81F5C12D81CFF
:1003F0005C12CF0B032A5908CF00591ADC16591E7C
:10040000DC12D91FDC12D00B0D2A5A08D000DA19E1
:100410005C17DA1D5C135A1E5C13D10B172A5B089C
:10042000D1005B1ADC175B1EDC13DB1FDC13D20B65
:100430001F2A5608D200D51B5D14D71F5D10D30BA1
:10044000272A5708D300D61BDD14D81FDD1008005B
:10045000C001DE080319DE035E184014DE1A4014E2
:100460004008C0015E1C4014DE1E4014C005C00CD4
:040470005E0C080016
:084000000F000300060006009A
:02400E00CC01E3
:10420000010003000300030003000200020002009B
:1042100002000000000000000000FF00FF00FF009F
:10422000000000000000000000000000000000008E
:104230000000C000C000C000C000FF00FF00FF0081
:104240000100C300F300CF00FF00C300F300CF0064
:10425000FF00C300F300CF00FF00FF00FF00FF00DE
:10426000FF00FF00FF00FF00FF00FF00FF00FF0056
:10427000FF00FF00FF00FF00FF00FF00FF00FF0046
:10428000FF00FF00FF00FF00FF00FF00FF00FF0036
:10429000FF00FF00FF00FF00FF00FF00FF00FF0026
:1042A000FF00FF00FF00FF00FF00FF00FF00FF0016
:1042B000FF00FF00FF00FF00FF00FF00FF00FF0006
:1042C000FF00FF00FF00FF00FF00FF00FF00FF00F6
:1042D000FF00FF00FF00FF00FF00FF00FF00FF00E6
:1042E000FF00FF00FF00FF00FF00FF00FF00FF00D6
:1042F000FF00FF00FF00FF00FF00FF00FF00AA001B
:00000001FF
